:020000040000FA
:0400000066303A2804
:040004000034003490
:08000800A000030EA100831209
:1000100005191128831601178312B2308100B1012E
:100020002C2883160113831203140B190310A80D37
:10003000A90DAA0DAB0DAC0DAC16FF302C02031DA3
:100040002C28FA302B02031D2C2832152A08AF0069
:100050002908AE002808AD008B100B11210E83007B
:06006000A00E200E0900B5
:0C007400203084008001840A80300402E7
:10008000031C3C285F2183160C30850587018312F1
:10009000850187010730990000309A0010308316DF
:1000A0008E008312603083168F0083120030831617
:1000B00091009F008312C830831681008312313073
:1000C0009000003083168C00831210308B00BD1B13
:1000D0006F2885196F286400851D6B28AC21A92124
:1000E00081018E018F010B118B100B108C018B176E
:1000F0008820321994204121B40B862803108519D9
:100100000314BA0DF0303A020319EC20DB217828F1
:1001100064003310B10A311F9328AC01AB01AA016E
:10012000A901A801B101080032110130B7008B13F9
:100130002030370783169B001C141A088312A40072
:100140001030370783169B001C141A088312A30073
:10015000A6000230A6060030370783169B001C1449
:100160001A088312A200A7000130A7068B17331CC0
:10017000BF2822090339A200A309A409A50924085C
:100180002F02031DE62823082E02031DD42822086F
:100190002D02031DE62801303702031DD4283E1826
:1001A000D4283E143F14792126082E02031DE62888
:1001B00027082D02031DE62801303702031DE5281C
:1001C0003E1CE5283E103F148A21E628B70A02307B
:1001D00037020318080097280130B600B400B500B4
:1001E000B70085018701B2139F218820B40B09292C
:1001F000031085190314BA0DF0303A02031931299E
:10020000B51F8501B51F8701B50B09299630B500CB
:100210003C21321DF5283211331C13292D090339D5
:10022000AD00AE09AF092F1CF5282D0830020319C7
:10023000F5282D08B0002E1EF5288B132030370727
:10024000BC002F08BB004A2110303707BC002E0825
:10025000BB004A2100303707BC002D08BB004A21F3
:100260008B1785018701A621B70AB6010230370234
:10027000031CF528A9210800013037020319962133
:1002800008003F1C08003F101030BC003E08BB00B7
:100290004A2108008B133B0883161C159A00831211
:1002A0003C0883169B0055309D00AA309D009C148D
:1002B00064009C1858291C1183128B1708008316A0
:1002C00000309B001C141A088312BD0083161030E6
:1002D0009B001C141A088312BE001430CA00CB0005
:1002E000CC00CD00CE00CF00D000D100D200D30092
:1002F00008000130BE00BD180230BD190230C00038
:10030000C100C200C300C400C500C600C700C800C9
:10031000C90008000830C000C100C200C300C4000A
:10032000C500C600C700C800C90008003809333935
:100330008500B80039093F398700B900080011303D
:100340008500B80013308700B9000800B801B90172
:1003500008003E1879210800B601B401B5013D1C22
:10036000B429BD01BD14C029BD1CB929BD013D156D
:10037000C0293D1DBE29BD01BD15C029BD013D14CB
:100380003D08B6006400C429C529C629C729C82963
:10039000B51B0516B51F0512B40BC229B50BC22932
:1003A0000310B60CB608031DC2290030BC003D087E
:1003B000BB004A21080054080E02031C051603184E
:1003C000051255080E02031C8516031885125608DF
:1003D0000E02031C05140318051057080E02031C17
:1003E00085140318851058080E02031C871403187F
:1003F000871059080E02031C0715031807115A0825
:100400000E02031C0714031807105B080E02031CDE
:100410008716031887125C080E02031C07160318C0
:1004200007125D080E02031C8715031887118F0839
:10043000031908008F0185018701401C272AFF301E
:10044000D400CA0B682AC001C0140A30D400C01CF2
:10045000342ACA0B682A1E30CA00D40F682AD40373
:10046000C00140151430DE00401D5B2ADE0B682AF7
:100470003030DE00FF30D400D500D600D700D800E1
:10048000D900DA00DB00DC00DD00CA0B682A853009
:100490005F07DF00CA0088303D19FF30BD19FF300B
:1004A000D400D500D600D700D800D900DA00DB0090
:1004B000DC00DD00682AC01D632ACA0B682A0A30E6
:1004C000CA00D40B682AD4011930CA00C001682AB6
:1004D000411C722AFF30D500CB0B8D2AC101C114FB
:1004E0000A30D500C11C7D2ACB0B8D2A0F30CB00E2
:1004F000D50F8D2AD503C1014115411D802A8D2AB2
:10050000C11D882ACB0B8D2A0B30CB00D50B8D2A31
:10051000D5011430CB00C1018D2A421C972AFF302F
:10052000D600CC0BB22AC201C2141930D600C21CAC
:10053000A22ACC0BB22A0A30CC00D60FB22AD6039C
:10054000C2014215421DA52AB22AC21DAD2ACC0BFA
:10055000B22A0930CC00D60BB22AD6011430CC0016
:10056000C201B22A431CBC2AFF30D700CD0BD72AC8
:10057000C301C3140A30D700C31CC72ACD0BD72A26
:100580000F30CD00D70FD72AD703C3014315431D22
:10059000CA2AD72AC31DD22ACD0BD72A0830CD00AC
:1005A000D70BD72AD7011430CD00C301D72A441C5A
:1005B000E12AFF30D800CE0BFC2AC401C4140F304E
:1005C000D800C41CEC2ACE0BFC2A0F30CE00D80F6A
:1005D000FC2AD803C4014415441DEF2AFC2AC41D7B
:1005E000F72ACE0BFC2A0D30CE00D80BFC2AD801FE
:1005F0001430CE00C401FC2A451C062BFF30D90064
:10060000CF0B212BC501C5141430D900C51C112BEB
:10061000CF0B212B1B30CF00D90F212BD903C501C4
:100620004515451D142B212BC51D1C2BCF0B212B34
:100630000B30CF00D90B212BD9011430CF00C501CD
:10064000212B461C2B2BFF30DA00D00B462BC6018A
:10065000C6140F30DA00C61C362BD00B462B0F30D9
:10066000D000DA0F462BDA03C6014615461D392B9A
:10067000462BC61D412BD00B462B0730D000DA0B82
:10068000462BDA011430D000C601462B471C502BF4
:10069000FF30DB00D10B6B2BC701C7140A30DB0026
:1006A000C71C5B2BD10B6B2B0F30D100DB0F6B2BDF
:1006B000DB03C7014715471D5E2B6B2BC71D662B40
:1006C000D10B6B2B0C30D100DB0B6B2BDB0114300F
:1006D000D100C7016B2B481C752BFF30DC00D20BFF
:1006E000902BC801C8140F30DC00C81C802BD20B23
:1006F000902B0A30D200DC0F902BDC03C801481588
:10070000481D832B902BC81D8B2BD20B902B0630B2
:10071000D200DC0B902BDC011430D200C801902BEE
:10072000491C9A2BFF30DD00D30BB52BC901C9142E
:100730000A30DD00C91CA52BD30BB52B1430D30018
:10074000DD0FB52BDD03C9014915491DA82BB52BBC
:10075000C91DB02BD30BB52B0B30D300DD0BB52B44
:0C076000DD011430D300C901B52B0800E6
:084000000500030006000900A1
:02400E00CC33B1
:10420000010078007A007C007E007B0079007F004E
:104210007D007A0078007E007C00FF00FF00FF0038
:104220000000F200F600FA00FE00F200F600FA00CC
:10423000FE00F200F600FA00FE00FF00FF00FF00A3
:10424000010005000500050005000900090009003E
:1042500009000D000D000D000D00FF00FF00FF0024
:10426000FF00FF00FF00FF00FF00FF00FF00FF0056
:10427000FF00FF00FF00FF00FF00FF00FF00FF0046
:10428000FF00FF00FF00FF00FF00FF00FF00FF0036
:10429000FF00FF00FF00FF00FF00FF00FF00FF0026
:1042A000FF00FF00FF00FF00FF00FF00FF00FF0016
:1042B000FF00FF00FF00FF00FF00FF00FF00FF0006
:1042C000FF00FF00FF00FF00FF00FF00FF00FF00F6
:1042D000FF00FF00FF00FF00FF00FF00FF00FF00E6
:1042E000FF00FF00FF00FF00FF00FF00FF00FF00D6
:1042F000FF00FF00FF00FF00FF00FF00FF00DD00E8
:00000001FF
